:1000000089C300000C947A2FA2C30000A0C3000093
:100010009EC300009CC300009AC3000098C3000068
:1000200096C3000094C300000C94B02D0C94982E3D
:100030000C94652D8CC300008AC3000088C30000A7
:1000400086C3000084C3000082C3000080C3000098
:100050007EC300000C948C2D7AC3000078C300008E
:1000600076C3000074C3000072C3000070C30000B8
:100070006EC300006CC300006AC3000068C30000C8
:1000800066C3000064C3000062C3000060C30000D8
:100090005EC300005CC300005AC3000058C30000E8
:1000A00056C3000054C3000052C3000005010902FA
:1000B000A10185020901A1000509190129081500FE
:1000C0002501950875018102050109300931158165
:1000D000257F95027508810609381581257F9501D0
:1000E00075088106050C0A38021581257F95017572
:1000F000088106C0C005010980A101850319012AF4
:10010000B700150126B700950175108100C0050CD8
:100110000901A101850419012AA002150126A002E6
:10012000950175108100C00660FF0961A101096297
:10013000150026FF00952075088102096315002629
:10014000FF00952075089102C005010906A101056F
:100150000719E029E7150025019508750181029529
:1001600001750881010507190029FF150026FF0008
:100170009506750881000508190129051500250156
:10018000950575019102950175039101C00000006C
:10019000000000000000000000000000000000005F
:1001A000000000000000000000000000000000004F
:1001B000007E0F00D4FFFFFFC700000078000000A2
:1001C00000000000002A2B280000000000000000B2
:1001D000000000000000000029000000002C1E3478
:1001E00020212224342627252E362D3738271E1F7E
:1001F000202122232425263333362E37381F0405A9
:10020000060708090A0B0C0D0E0F10111213141516
:10021000161718191A1B1C1D2F3130232D350405F4
:10022000060708090A0B0C0D0E0F101112131415F6
:10023000161718191A1B1C1D2F3130354C09025B7B
:1002400000030100A0FA09040000010301010009F4
:100250002111010001224400070581030800010962
:100260000401000203000000092111010001222203
:100270000007058203200001070503032000010990
:100280000402000103000000092111010001227B8A
:10029000000705840320000112010002000000088D
:1002A00010CB56210002010203011C0376006900F5
:1002B00061006C003A0066003600340063003200D2
:1002C00062003300630000001E034E0079007100DD
:1002D000750069007300740020005200650076000C
:1002E0002E002000320000000E034B006500650068
:1002F000620069006F0000000403090435001E005D
:100300001F002000210022002B0014001A0008000A
:1003100015001700290004001600070009000A0054
:10032000E1001D001B000600190005002552E00039
:10033000E200E30023522C002A00270026002500BB
:10034000240023004C00130012000C0018001C00B5
:10035000340033000F000E000D000B0028003800A1
:1003600037003600100011004F00520051005000BD
:1003700024522C0035001E001F0020002100220006
:100380002B0014001A00090013000A0029000400C1
:100390001500160017000700E1001D001B000600F5
:1003A000190005002552E000E200E30023522C0072
:1003B0002A00270026002500240023004C003300DB
:1003C0001C0018000F000D00340012000C00080083
:1003D00011000B00280038003700360010000E0016
:1003E0004F0052005100500024522C0035001E00D6
:1003F0001F002000210022002B00340036003700AF
:1004000013001C00290004001200080018000C0052
:10041000E100330014000D000E001B002552E00027
:10042000E200E30023522C002A00270026002500CA
:10043000240023004C000F00150006000A000900EC
:1004400038001600110017000B00070028001D00DF
:1004500019001A00100005004F0052005100500012
:1004600024522C0035021E021F0220022102220209
:1004700035021E021F022002210222024C003A0015
:100480003B003C003D003E0005784000410042003A
:1004900043004400010001000100010001000100CF
:1004A0002A00270226022502240223024C002702EA
:1004B0002602250224022302310230022F022E02DC
:1004C0002D023F0001004D004A0064023202450047
:1004D000AE00A900AA00AB000100010035001E001B
:1004E0001F0020002100220035001E001F002000F8
:1004F000210022004C003A003B003C003D003E0041
:10050000010040004100420043004400010001009E
:1005100001000100010001002A002700260025003B
:10052000240023004C00270026002500240023007F
:10053000310030002F002E002D003F0001004E0042
:100540004B00640032004500AE00A900AA00AB00D9
:10055000010001003A003B003C003D003E003F002E
:100560000100007C4278437846784578010001001C
:100570000100807481741570010001000100010008
:100580000100010001000100010001000100010063
:100590004500440043004200410040004C0001007F
:1005A00049784A7847784878010001004252415220
:1005B000405214700100010001000100010001001F
:1005C000010001000100010001000100FD377A581F
:1005D0005A000004E6D6B4460200210116000000CD
:1005E000742FE5A3E003B201085D003D888986D33E
:1005F000DC0AE842C3249258425AFA4B42162C5F56
:10060000542BA3199BCDF09E3ED52B7388208A27AF
:1006100002C28C6C91863337C68276CB812B45B073
:100620004557660343EA9B6B19E8B1AAA5E31F2C63
:1006300065784B4034F572DD554C0E88976FFB9210
:100640000FB4A5F05BB19A2B1D54928E8272F648BE
:10065000E7B4799F489284ADB1C6FC79939A8D1C1A
:1006600035FF1B43F6C6C36EBA331667230739003E
:1006700080DCF0C90C81E00A7D63DD01534C5B95A1
:10068000B69BDD20F18041788D582E31A49DE6E4A3
:1006900022C3AEFD3C42DB72E04C0613E4B985296F
:1006A000FF5AE82552FB2F1DAE76F50CE6A9333E26
:1006B000C260D50808F250A7490CB73F7F5CCCBB9D
:1006C0008B1564DEBF6F0059C9DDAAEC69D00951F2
:1006D000F1D362269E135492CC3819E51A9CEAD3C2
:1006E00022865F6703DF3AED5FB76A10E5AD968D4E
:1006F0004D7F0000B6C38E336581AEE60001A402D3
:10070000B3070000B4239031B1C467FB02000000BE
:100710000004595A11241FBECFEFDAE0DEBFCDBF6F
:1007200011E0A0E0B1E0E4E7F4E602C005900D922C
:10073000A43CB107D9F723E0A4ECB1E001C01D92BD
:10074000A23FB207E1F70E9469260C94C53158CC4C
:100750009C019A9581159F4118F5F32FF270EE27B1
:10076000832F8170732F74706627532F587044271E
:1007700034FF0CC08295807FEF2B09F08062672BDD
:1007800009F08064452B69F080680895EF2B09F02B
:100790008260672B09F08460452B19F0886008950A
:1007A00080E00895CF93DF93EB01D2DFFE0109953E
:1007B000DF91CF910895982F92959F7024E0911129
:1007C00002C020E0982F892F86958695811511F01B
:1007D0002E5F982F892F8695820F08958093A70307
:1007E00008958093A803089521E030E001C0220F0E
:1007F0008A95EAF78091A803822BF3CF21E030E0BD
:10080000A90102C0440F551F8A95E2F7CA018095DD
:100810009091A8038923E5CF292F9A3090F586304F
:1008200080F590E036E0239F800D911D1124282F44
:10083000277041E001C0440F2A95EAF723E096951E
:1008400087952A95E1F7FC01EE0FFF1FE80FF91FCE
:10085000E859FD4F20E030E070E05191DF01CB011D
:10086000022E02C0969587950A94E2F781708195D1
:100870008527842385278E932F5F3F4F23303105B3
:1008800061F70895292F9A3078F5863068F590E061
:1008900036E0239F800D911D1124682F677023E09F
:1008A000969587952A95E1F7FC01EE0FFF1FE80F5B
:1008B000F91FE859FD4F40E050E080E0219130E021
:1008C000062E02C0369527950A94E2F72170332749
:1008D000042E01C0220F0A94EAF7822B4F5F5F4F6C
:1008E0004330510559F7089580E008959091A80389
:1008F00021E030E0F90101C0EE0F8A95EAF7D90155
:1009000002C0AA0FBB1F6A95E2F7EA2B01C0220FB3
:100910004A95EAF7892F8E23E81303C0892F822B8B
:1009200060CF2095822F8923FBCF8091B0039091D7
:10093000AF03981301C008958F5F8770FACF90912D
:10094000AA03809589238093AA03282F2770211159
:1009500010C0891771F09091F10392FF0AC086953B
:10096000869586954BDF1092AA031092AC031092E5
:10097000AB0308959091A503982B9093A503089538
:10098000982F90958091A50389238093A5030895BE
:100990008091A403811531F01092A4031092AE034C
:1009A0001092AD030895803E9105D9F1C8F48133CA
:1009B000910509F482C048F48932910509F472C0A6
:1009C0008A32910509F480C0089589339105E9F0D0
:1009D00082389105D1F08533910509F45EC0089500
:1009E000843E9105D9F148F4823E910539F1833E68
:1009F000910549F181EE90E00895863E9105C9F197
:100A0000873E910509F43EC008952091F0032370BC
:100A1000211164C02091F10323FF14C089E290E00A
:100A200008952091F00320FD45C03091F10330FF7F
:100A300009C024FD24C083EE90E008952091F003C6
:100A400022FDF7CF08952091F00322FD44C030919C
:100A5000F10330FD43C024FFF5CF11C02091F10315
:100A600021FFF0CF8091F00384FD09C087EE90E074
:100A700008952091F00323FFE5CF24FFF7CF80E016
:100A800090E008952091F00323FD2BC03091F103F5
:100A900031FFE1CF84EE90E008952091F00325FF2F
:100AA000D1CFBCCF2091F00325FD1EC02091F103D2
:100AB00023FFC8CF89E390E008952091F00326FF3B
:100AC000C1CF8AE290E008952091F00326FFBACFCB
:100AD00081E390E0089582EE90E0089580EE90E04A
:100AE000089586EE90E0089585E390E00895909152
:100AF000F00392FF10C041E0282F2471243009F048
:100B000040E031E0282F2871283009F030E0431709
:100B100011F02CE0822793FF10C041E0282F2471B0
:100B2000243109F040E031E0282F2871283109F004
:100B300030E0431711F02CE082273091F10330FFB1
:100B400010C051E0282F2171213009F050E041E020
:100B5000282F2871283009F040E0541711F029E0BF
:100B6000822731FF10C041E0282F2171213109F087
:100B700040E031E0282F2871283109F030E0431798
:100B800011F029E0822794FD877E08951F93CF936B
:100B9000DF9309DFEC01811522E5920708F052C0CE
:100BA000811540E5940708F0CDC0803E910520F501
:100BB0008D3C910508F0A1C0883A910570F4853A02
:100BC000910508F097C081309105B9F10497813AF9
:100BD000910598F1C0E0D0E030C0885A91094B9758
:100BE000C8F7C85AD0E0CC0FDD1FC95ADE4F0990B4
:100BF000D881C02DD46421C0811550E49507B0F48C
:100C0000C11580E2D80708F0B3C0C83ED105A8F0EE
:100C1000CE019A9581159F41E8F68D2F68DF182F38
:100C2000CE019927C0DEEC01D12B07C09927BBDE8E
:100C3000CC27DF70C82BD92BD06ACE01DF91CF91A2
:100C40001F910895803842E59407C8F5803652E533
:100C5000950708F05BC0C03482E5D807D0F4C032F5
:100C600092E5D90708F04BC08C2F8695869520E237
:100C7000829FC0011124C37021E030E0A90102C0AD
:100C8000440F551FCA95E2F7EA01C82BD92BDD683E
:100C9000D4CF8C2F86958695877050E2859FC001B2
:100CA0001124C37021E030E0A90102C0440F551F98
:100CB000CA95E2F7EA01C82BD92BDC68BECF803C8D
:100CC00052E5950758F48F71C03AD245A0F590E0EF
:100CD000982F8827EC01C46FD06AAFCF805C924513
:100CE000809708F077CFDC2FCC27CC27DF71C06F3F
:100CF000D06AA3CFA497D064A0CFD0659ECFCF7188
:100D0000D0E0DC2FCC27C16FD06A97CF869586952F
:100D1000877020E2829FC0011124C37021E030E07F
:100D2000A90102C0440F551FCA95E2F7EA01C82B7A
:100D3000D92BDA6882CFDBDEC82FD0E0DC2FCC27BE
:100D4000D0627BCF8F71D3DE93E0CC0FDD1F9A95FD
:100D5000E1F7CC27DF70282F30E084FF05C050E199
:100D6000859F900111243327C22BD32BD06965CFE7
:100D70008D2F8F71BCDE182FCE01992714DEEC0168
:100D8000D12BDECF80E00895F894E82FE295EF7044
:100D9000F0E041A18F7021E030E0B90102C0660FA0
:100DA000771F8A95E2F7CB01962F9095942391A314
:100DB00092A1892B82A378940895A0E0B0E0E3EE9D
:100DC000F6E00C949330883080F581112FC090911B
:100DD00080009F7D90938000209186003091870055
:100DE000A82FB0E00E94253127E030E040E050E03D
:100DF0000E94F63069017A01809186009091870007
:100E00006CE070E00E94CF306217730798F0C90160
:100E100069E070E00E94CF3070938B0060938A008D
:100E2000CDB7DEB7E8E00C94AF3087E0909180005A
:100E30009062D0CF809186009091870000918600CB
:100E4000109187002091860030918700C6E0D0E0A5
:100E5000BE010E94CF30C60ED71EE11CF11C85E0FA
:100E6000CC0CDD1CEE1CFF1C8A95D1F7C801BE011D
:100E70000E94CF3040E050E0260F371F411D511D2A
:100E8000C701B6010E94F63069017A01E09186003F
:100E9000F0918700CA01B9010E94C0309B01AC01EA
:100EA000DF010E9434319B01AC01C701B6010E94F1
:100EB000C0302FE096958795779567952A95D1F75D
:100EC00020918600309187002617370718061906EB
:100ED00008F0A2CF60918600709187009DCF883086
:100EE00008F087E0209193022770982F990F990FAF
:100EF000990F922B9093930221E0983008F420E010
:100F00009091930220FB90F99093930256CF811514
:100F10002CE7920741F42091330230913402232BC5
:100F200011F480E090E00895EDE1F3E080E090E0DE
:100F300067E275E24AE455E22CEB35E2778366839B
:100F400051874087338722879787868701967096D7
:100F50008830910599F70895FC01848186238111D9
:100F60000AC082818115B9F06823908593FF05C07E
:100F700081E061110FC080E00895282F22952F7025
:100F80008F70282B962F92959F706F70962B81E013
:100F90002913F1CF089581E008950F931F93CF9304
:100FA00001E010E0082E01C0000F0A94EAF7C0919A
:100FB000A3039C2F9023911115C09091AA0396959D
:100FC00096959695891306C01092AA031092AC03C9
:100FD0001092AB0309DCC027C093A303CF911F91EC
:100FE0000F9108950BDCF7CF282F35EB2303C001B9
:100FF000112497FF04C080589109892F08958058C3
:101000009F4FFBCF8091820280FD14C081FD14C0F0
:1010100082FD16C080918102811581F08E3180F4AD
:1010200020E5829FC00111246EE170E00E94E33050
:10103000862F089584E1089588E2089588E0089550
:1010400080E508958091820280FD17C081FD17C060
:1010500082FD19C080918002811599F0883298F440
:1010600028E0829FC001112468E270E00E94E33012
:101070006115710551F0862F089562E0FCCF64E0A0
:10108000FACF61E0F8CF68E0F6CF81E00895FA0189
:10109000309709F00995089580915202811569F001
:1010A000E0915E02F0915F02309739F00190F0819B
:1010B000E02D309711F00995089580E00895A3E0A0
:1010C000B0E0E5E6F8E00C9499309C018091F401E1
:1010D0009091F50182179307B1F03093F5012093B9
:1010E000F401E0915E02F0915F02309761F00084BC
:1010F000F185E02D309739F083E089833B832A83A3
:10110000CE01019609952396E2E00C94B530A3E058
:10111000B0E0EDE8F8E00C9499309C018091F20188
:101120009091F30182179307B1F03093F30120936C
:10113000F201E0915E02F0915F02309761F000846D
:10114000F185E02D309739F084E089833B832A8351
:10115000CE01019609952396E2E00C94B530A8ECF7
:10116000B1E0EFEF90E02D91821751F0EF3F19F4CD
:10117000211101C0E92F9F5F9630A9F7EF3F09F4D5
:1011800008950E2E000CFF0BEA53FE4F8283089544
:10119000E8ECF1E09191891302C0DF011E9291E029
:1011A000EE3CF907B9F708958091010108952FB732
:1011B000F8948091EE019091EF01A091F001B0912F
:1011C000F1012FBF0895962F2091F10322FF0EC049
:1011D000682F660F660F660F692B6093AA0304DB06
:1011E000E6DF9093AC038093AB030895FDCA909122
:1011F000A403292F2823211559F080958923809352
:10120000A403811531F0D3DF8093AD039093AE0337
:10121000089580E090E0F8CFCADF209185023091F8
:101220008602232B211521F0809322029093230222
:101230002091870230918802232B211521F0809381
:10124000200290932102E0915E02F0915F023097BC
:1012500059F00680F781E02D309731F082E08093DD
:10126000830283E892E009950895611509F441C06D
:10127000E3E3E80FE33148F4F0E0E953FE4C0C946B
:101280001831C0DE819580938602C6CFBBDEFBCFCE
:10129000B9DE819580938502F8CFB4DEFBCFD2DE34
:1012A00080938702F2CFCEDE8195FACFCBDE819597
:1012B00080938802EACFC6DEFBCF815D990B21E0E7
:1012C00030E001C0220F8A95EAF780918402822BD8
:1012D00080938402DACF80918202816080938202BF
:1012E000D4CF809182028260F9CF809182028460A3
:1012F000F5CF409185028D3C59F48091860287FF9D
:101300000DC010928602411559F41092810208C056
:101310008E3C81F48091860218169CF3411581F071
:101320008091870290918802892B8111AECF109213
:101330008002ABCF8F3C41F447FFF0CF1092850283
:10134000809186028115E0CF803D19F41416B4F324
:10135000E5CF90918702893D29F41916FCF6109289
:101360008702DCCF8A3D19F497FFD8CFF8CF909150
:1013700088028B3D29F497FFD1CF10928802CECFFF
:101380008C3D19F41916CCF3C9CF9FE2980F983011
:1013900090F4815D990B21E030E0B90102C0660F45
:1013A000771F8A95E2F7CB0180959091840289237B
:1013B00080938402B3CF8D3D31F4809182028E7F81
:1013C00080938202ABCF8E3D21F4809182028D7F8B
:1013D000F7CF8F3D09F0A2CF809182028B7FF0CFB3
:1013E0002FB7F8946091EE017091EF018091F001B8
:1013F0009091F1012FBF08950F931F938091520296
:10140000811521F0EDDF1F910F910895E9DF009123
:101410005402109155022091560230915702600FEC
:10142000711F821F931FEFCFCF92DF92EF92FF9237
:10143000CF93DF93D82FC92FC0901703D0901803F4
:10144000E0901903F0901A03CBDF6C197D098E0927
:101450009F09643F71408105910510F1C1DF6B0167
:101460007C0182E390E0A0E0B0E0C0921C02D09248
:101470001D02E0921E02F0921F02809318029093C8
:101480001902A0931A02B0931B02D0931503C093C4
:101490001603DF91CF91FF90EF90DF90CF900895EA
:1014A00084EF91E0A0E0B0E0E0CF87E797E790938A
:1014B00001088093000888E19AE00FB6F894A89597
:1014C000809360000FBE90936000FFCF0895FC01F1
:1014D0009B018091E4019091E5018617970740F008
:1014E000672B29F48091E8008E778093E800C9018A
:1014F00040E0009741F4411106C08091E80082FF6E
:101500002FC080E00895209135022115A9F12530E2
:10151000A9F12091E80023FD2DC02091E80022FDD3
:10152000ECCF2091E80020FFE4CF3091F300209130
:10153000F200009719F02830310558F041E02830CA
:10154000310509F040E02091E8002E772093E80073
:10155000D0CF41914093F10001972F5F3F4FE9CFEA
:1015600080913502811541F0853041F08091E8008D
:1015700083FFC3CF81E0089582E0089583E008955A
:101580008091DE0187FF13C08091E80082FF06C0D2
:101590008091E8008B778093E80008958091350270
:1015A0008111F2CF0895809135028115D9F3809190
:1015B000E80080FFF8CF8091E8008E77ECCF209193
:1015C000E4003091E50095E6A9012091EC00822F1E
:1015D000817020FF06C08091E80080FF06C080E097
:1015E00008952091E80022FD1AC0809135028115EE
:1015F00089F0853089F08091EB0085FD0FC0209146
:10160000E4003091E50042175307F9F29A95E1F6AC
:1016100084E0089582E0089583E0089581E00895CC
:10162000E8EDF0E080818E7F80831092E2001092DE
:10163000DA001092E100A0EEB0E08C9181608C9312
:1016400080818F77808319BCA7EDB0E08C918E7F6D
:101650008C9380818F7E80831092DD010895E091CC
:101660005E02F0915F02309739F00284F385E02D3D
:10167000309711F060E209950895FC01AC014B5FD1
:101680005F4F8FEF61E39191892728E030E0982F39
:10169000990F87FF09C0892F862721503040B9F75D
:1016A000E417F50781F70895892FF7CF982F9093C6
:1016B000E900891771F07091EC002091ED005091D4
:1016C000F00021FD09C09F5F973089F78093E90002
:1016D0000895762F242F50E03091EB003E7F309319
:1016E000EB003091ED003D7F3093ED003091EB0049
:1016F00031603093EB007093EC002093ED00509339
:10170000F0002091EE0027FDDECF0895A0E0B0E0CC
:10171000ECE8FBE00C949330C8EDD0E088818F7E3C
:101720008883E7EDF0E080818160808384E082BF80
:1017300081E08093DD0188818E7F888302EE10E056
:10174000F80110821092DA0081EEC82ED12CF60139
:10175000108288818F7788838881806888838881D8
:101760008F7D888319BC109235021092DC01109293
:101770000C021092DB0190EEE92EF12CF701808132
:101780008B7F808388818160888342E060E080E095
:101790008DDFF60180818E7F8083F80180818160FA
:1017A0008083808188608083F70180818E7F808341
:1017B000888180618883CDB7DEB7E8E00C94AF30D4
:1017C000E091B0039091AF0327E0E91302C080E0FD
:1017D0000895AE2FB0E02E9FF0011124EF54FC4F7E
:1017E0003181361306C03081381303C0358134137C
:1017F00004C0FD013196E770E8CF81E008950F93B2
:101800001F93CF93DF938B01EA01909135029430BF
:1018100051F58093E9008FEF9091E80095FD06C0A7
:1018200095ED9A95F1F700008A95B1F78091E8005F
:1018300085FF19C0C4DE811111C08091E80085FDCB
:1018400006C08091E8008E778093E800F3CFF8011E
:1018500081918F018093F100219779F78091E800C1
:101860008E778093E800DF91CF911F910F910895BB
:10187000792F603229F440E250E0682F82E0BFCF38
:101880000895CF93DF93D82FC92F48E050E0682FF9
:10189000792F81E0B4DF88E0ED2FFC2FA6EEB1E0D8
:1018A00001900D928A95E1F7DF91CF910895BC01E7
:1018B00046E050E084E0A3CFBC0143E050E084E088
:1018C0009ECFA0E0B0E0E7E6FCE00C949130F82E6B
:1018D000E92EB62EA72E8A018091D8019AE0C92E52
:1018E000D12C8A3018F0CC24C394D12CC1E0D0E0A4
:1018F0006B2D7A2D8F2D9E2DF8010995811116C023
:101900002196CC16DD0694F0CC9FC001CD9F900DA2
:10191000900D112420E030E045E34A95F1F70000F6
:101920002F5F3F4F28173907B9F7E2CFCDB7DEB7A2
:10193000EAE00C94AD30CF93DF93C1E0D0E001C07A
:10194000CC0F8A95EAF76C2F83E090E00E949031EB
:101950008C2F0E94EE03DF91CF910895FC016081EE
:1019600086E090E00C9490318091930280FD11C04C
:10197000816080939302813019F489E0809393020F
:1019800083E992E0EBDF80919302869586958695B8
:1019900014CA08951F93CF93DF93962F122F632FAE
:1019A0008630D8F49A30C8F44630B8F4C42FD0E06A
:1019B000CC0FDD1F2CE0929FC00DD11D112498E7A4
:1019C000899FC00DD11D1124CE0189960E949031AE
:1019D000612FCE018A960E949031DF91CF911F91A5
:1019E00008959091F10392FB222720F9281779F0AE
:1019F00080FB92F99093F1036091F0037091F103F1
:101A000084E090E00E94AA3182E00C949F04089543
:101A1000CF93DF93C091A5038091A903C82B809138
:101A2000A4038115F1F0C3DB2091AD033091AE0327
:101A3000821B930B8838934110F00E94C804D09108
:101A4000A40320E088EC91E0FC0130810196311183
:101A50002F5F31E08E3C9307B9F721110E94C80433
:101A6000CD2B8091990280958C2390919802892B9F
:101A70008093C60148E050E060E672E086EC91E0B9
:101A80000E944731892BB9F088E0E6ECF1E0A0E64E
:101A9000B2E001900D928A95E1F7E0915E02F0913B
:101AA0005F02309741F00280F381E02D309719F00A
:101AB00086EC91E00995DF91CF910895CF93109234
:101AC000A503C6E0E8ECF1E0DF018C2F1D928A95BA
:101AD000E9F780E090E0F3DA80E090E018DB109224
:101AE000A90396DFE3E8F2E0DF011D92CA95E9F76A
:101AF0001092810210928002109282028DDBCF91AF
:101B00000895DCDF2FEF84E39CE02150804090407B
:101B1000E1F700C0000088E19AE00FB6F894A895BC
:101B2000809360000FBE90936000FFCFAAE2B0E008
:101B3000ECE9FDE00C9498308EED91E0FC0101960B
:101B40002091F100208321E0863E9207B9F7809131
:101B5000DF01893009F457C0C8F4823009F4B2C0FB
:101B6000833009F482C0813081F18091E80083FFE5
:101B7000E6C08091DE019091DF019A3008F0DFC06D
:101B8000E92FF0E0E652FE4C0C9418318A3009F44B
:101B900089C08B3051F78091DE01813231F780911D
:101BA000E2019091E301892B01F78091E800877FA2
:101BB0008093E800E5DC81E09091E001911101C0A3
:101BC00080E0809302017ADFD0CF8091DE01813AFC
:101BD00061F68091E800877F8093E8008091E201C0
:101BE0009091E301892B59F060E080E090E070E093
:101BF0006EDC8091E8008B778093E800B6CF68E0D8
:101C000086EE91E0F4CF8091DE01813209F0ADCF14
:101C10008091E2019091E3018D7F892B09F0A5CF9E
:101C20008091E800877F8093E8008091E80082FF40
:101C300017C09091F3008091F200029731F48091E7
:101C4000F100813011F0863021F48091F100809311
:101C500001018091E8008B778093E80091DC85CFCB
:101C6000809135028111E1CF80CF8091DE01813AF0
:101C700009F07BCF8091E2019091E301892B09F07B
:101C800074CF8091E800877F8093E8008091E8001E
:101C900080FFFCCF809102018093F1008091E800E9
:101CA0008E77DACF8091DE01813209F05ECF8091AC
:101CB000E800877F8093E80063DC8091E1018093F6
:101CC000000153CF8091DE01813A09F04ECF80911F
:101CD000E800877F8093E8008091E80080FFFCCFD8
:101CE00080910001D9CF803889F0823841F5809108
:101CF000E2018F70873018F58093E9008091EB0046
:101D000085FB882780F91092E90006C080910C02BB
:101D1000880F9091DB01892B9091E800977F909339
:101D2000E8008093F1001092F1008091E8008E7736
:101D300023C0811116C08091E001813009F18091AA
:101D4000E80083FF0AC08091E800877F8093E80065
:101D50008091EB0080628093EB00AA96E3E00C9404
:101D6000B430823061F78091E001811581F01092EA
:101D7000E9008091E800877F8093E80001DCDFCFF5
:101D800081E0933009F080E080930C02F0CF8091E5
:101D9000E2018F702FEF280F263088F68093E9003C
:101DA0002091EB0020FFE3CF933031F48091EB00E2
:101DB00080628093EB00DBCF9091EB009061909379
:101DC000EB0021E030E0A90102C0440F551F8A95C5
:101DD000E2F74093EA001092EA008091EB008860FD
:101DE000E8CF8111ACCF1091E0011F778091E30023
:101DF0008078812B8093E3008091E800877F809337
:101E0000E800BEDB8091E80080FFFCCF8091E3001A
:101E100080688093E30083E0111101C082E0809329
:101E200035028DCF8058823008F089CF8091E00153
:101E30009091E1018C3D53E0950791F583E08A8311
:101E40008AE289834FB7F894DE01139620E03EE0E2
:101E500051E2E32FF0E050935700849120FF03C03C
:101E600082958F703F5F8F708A30C0F0895C90E000
:101E70008D939D932F5F243161F74FBF8091E800D0
:101E8000877F8093E8006AE270E0CE0101961FDB55
:101E90008091E8008B778093E80051CF805DE7CF99
:101EA000292F33272330310509F44EC078F521302E
:101EB000310509F488C08BE590E0EDE3F2E02230D3
:101EC000310509F03CCF2091E800277F2093E800FE
:101ED0002091E4013091E5018217930708F49C01F9
:101EE00040E02115310509F073C0411171C08091A6
:101EF000E80082FDCDCF80913502811549F2853011
:101F000039F28091E80083FFF2CFC2CF8091E201E5
:101F10009091E3012132310509F446C022323105A6
:101F200009F00DCF8330910508F009CFFC01EE0FC9
:101F3000FF1FE25CFE4F0190F081E02D855C9E4F1B
:101F4000DC018C9190E010C09C013327823021F19C
:101F50002330310568F4232BB9F4E8EFF2E0E49183
:101F60008E2F90E0E8EFF2E0009709F4E8CEABCFD7
:101F70002330310509F0E3CEEAEAF2E0E4918E2F56
:101F800090E0EAEAF2E0F0CFE8EEF2E0E4918E2FA2
:101F900090E0E8EEF2E0E8CFE8ECF2E0E4918E2F9A
:101FA00090E0E8ECF2E0E0CF8330910508F0C7CE96
:101FB000FC01EE0FFF1FEC5BFE4F0190F081E02D66
:101FC00089E090E080CF82E190E0E8E9F2E07BCF29
:101FD00080913502811509F45BCF853009F458CF23
:101FE0008091E80083FD54CF8091E80082FD7FCF8F
:101FF0008091E80080FF75CF9091F3008091F2000E
:102000002115310519F08830910550F041E008970D
:1020100009F040E08091E8008E778093E80061CF7E
:1020200044914093F1003196215031090196E8CF57
:10203000803809F084CE8091E800877F8093E800A3
:102040008091DC018093F10070CE811178CE1091E7
:10205000E001123008F073CE8091E800877F809312
:10206000E8001093DC018CDA1115D9F084E080933C
:10207000350242E061EC81E019DB42E261EC84E090
:1020800015DB42E261EC82E011DB42E260EC83E0CE
:102090000DDB80913502843051F482E0809303019E
:1020A0004ECE8091E30087FDE1CF81E0E0CF81E07B
:1020B000F5CFCF93C82F8115A9F08238A9F40E94DB
:1020C0004C0881FD0FC089E34AD8A2DC2FEF37EE20
:1020D00083E0215030408040E1F700C0000089E3F8
:1020E00057D896DCCF910895833891F40E944C081C
:1020F00080FDF8CF83E533D88BDC9FEF21EE34E011
:10210000915020403040E1F700C0000083E5E8CF67
:10211000843891F40E944C0882FDE4CF87E41FD8F4
:1021200077DC8FEF91EE24E0815090402040E1F782
:1021300000C0000087E4D4CF8CEF8C0F813A68F4A4
:10214000E8ECF1E08EEC91E02191C217A9F18E1735
:102150009F07D1F78C2F03D8C4CF80E28C0F883033
:1021600048F4C77081E001C0880FCA95EAF70E9461
:10217000BA04B7CF8BE58C0F833038F42C2F245260
:10218000330BC9010E945F08ADCFE8E5EC0FEB31DE
:1021900050F4F0E0EE0FFF1FE357FE4F8081918176
:1021A0000E9487089FCF83E38C0F833108F09ACF7A
:1021B00061E08C2F5AD896CF8C2F0E94C80828DC5B
:1021C000C9CFCF93DF93EC01805E9109089720F08F
:1021D0006BE671E1209711F46FE571E1CE010E9489
:1021E000D2038C2F66DFDF91CF910895811509F41A
:1021F0004FC0823861F40E944C0881FF49C089E3D6
:102200000E94AF0805DC89E30E94C80801CC83382E
:1022100051F40E944C0880FF3BC083E50E94AF0848
:10222000F7DB83E5F1CF843851F40E944C0882FF3C
:102230002FC087E40E94AF08EBDB87E4E5CF9CEF7B
:10224000980F913A08F390E2980F983050F4877005
:1022500091E001C0990F8A95EAF7892F0E94C00486
:10226000D5CF9BE5980F933020F480E090E00C945C
:102270005F0898E5980F9B3120F480E090E00C9483
:10228000870893E3980F933118F460E00C943509B4
:1022900008951F93CF93DF93182FEB010ADF209748
:1022A00031F4812FA3DFDF91CF911F9108958FE942
:1022B0009FE00197F1F700C000002197F0CF811552
:1022C00019F00E94BA04A4CB0895811519F00E9458
:1022D000C0049ECB0895811531F09091A903892BFC
:1022E0008093A90395CB0895811539F0809590913D
:1022F000A90389238093A9038BCB0895809194022D
:10230000811521F082E2F0DF109294020895CF93BC
:10231000DF93EC014A855B856E857F850E944708C7
:102320009B8190958091A90389238093A9038C8137
:102330000E94C0046DDB86E0FE0111928A95E9F7E8
:10234000DF91CF910895CF93DF93EC018D8181FDD3
:1023500013C082608D838091A9039B81892B809318
:10236000A9038C810E94BA0453DB488559856E8588
:102370007F85CE010E94470810929E0310929D0314
:102380008D8180FD02C0CE01C2DFDF91CF91089523
:102390001F93CF93DF93182FA0911303B0911403D1
:1023A000109709F448C0109216031092150310926A
:1023B0009902109298021696CD91DC911797CE0152
:1023C0009A9581159F4108F4D07ED1E0C11101C0DA
:1023D000D0E01996ED91FC911A97309731F01B9649
:1023E0006D917C9180E00995D823D11539F08CEF5F
:1023F0008C0F813A20F58C2F0E94C8081115A1F08E
:10240000E0911303F0911403808584FD0DC0809149
:102410001203811549F0808191819C01215031097D
:102420002F333E4708F400D8F3DA109214031092C9
:10243000130310921203DF91CF911F910895E8DAF0
:102440008C2FD4DEDBCFAFE0B0E0E9E2F2E10C9418
:102450008C30FE0131968AE0DF011D928A95E9F702
:102460008AE4E82E81E0F82E8F019FE4C92E91E0E6
:10247000D92E3F01AA24A394B12C35E5832E31E057
:10248000932EF70181917F018F3F09F43EC0F894AC
:10249000E82FE295EF70F0E021A18F70A50102C056
:1024A000440F551F8A95E2F7CA01922F982B91A3EA
:1024B00092A18095892382A3789400C0EFE4F1E093
:1024C00031E0512C21912F3F79F0A22FA295AF70CE
:1024D000A05EB0E08C9190E02F7002C0959587953A
:1024E0002A95E2F780FF7BC080E0582A330F8E16D2
:1024F0009F0641F7F70182918F3F11F00E94C406B9
:1025000050EA5A95F1F7D8015C920F5F1F4FCE1435
:10251000DF0409F0B6CF4AE050E0B3018FEF91E05D
:102520000E9447319C01892B41F08AE0F301AFEF13
:10253000B1E001900D928A95E1F700910A0210E056
:10254000075D1D4F232B09F44CC081E08093D70118
:102550000E94D7089093D6018093D50180915202B2
:10256000811509F498C07E01BBE0EB0EF11C85E0FB
:10257000F70111928A95E9F78091D8018A3008F025
:1025800054C04CE854E1B701C8019BD9811509F446
:1025900070C041E354E1B701C80193D9811509F432
:1025A00068C049E255E1B701C8018BD9811509F42A
:1025B00060C01092D8018091090290E045E050E09F
:1025C000B701875D9D4F0E94473121E02093D401E0
:1025D000892B09F041C02F96EFE00C94A830832F8F
:1025E00084CF8091D701811509F4B8CFE090D5014F
:1025F000F090D6010E94D7088E199F09059708F41C
:10260000ADCF45E050E06FEF71E0C8010E94473167
:10261000892B41F085E0EFEFF1E0D80101900D92B8
:102620008A95E1F71092D70199CFC090D201D0904E
:10263000D3010E94D7088C199D09843F914008F06E
:10264000A0CF8091D401811531F285E0D7011D9290
:102650008A95E9F71092D401A0910902B0E0A75D34
:10266000BD4F85E0FE013B9601900D928A95E1F702
:10267000B2CF8091D8018F3F39F40E94D708909350
:10268000D3018093D201DDCF8F5F8093D8018A3050
:1026900008F491CFF2CF85E0F801AFE3B2E001900A
:1026A0000D928A95E1F78FE392E00E943D0B8093B3
:1026B0003E02C0904402D0904502E0904602F09065
:1026C00047028091CE019091CF01A091D001B091AD
:1026D000D101C816D906EA06FB06B1F0C092CE01B8
:1026E000D092CF01E092D001F092D1010E94F00986
:1026F000C61AD70AE80AF90AC0925402D0925502C3
:10270000E0925602F0925702809148020E946F07B1
:1027100062CFA0E0B0E0EFE8F3E10C949230EC017E
:102720008881811509F1813009F045C089818130A6
:1027300051F48A81239660E570E0893311F060E0FE
:1027400070E0A7DDEDCF823021F48A812396B1DCE1
:10275000E7CF833021F48A81239648DDE1CF8430AE
:1027600041F022968111DCCFCDB7DEB7E9E00C94C1
:10277000AE308A81239620E030E09AE0682F6053E3
:10278000770BAB016A30710560F02115310551F30B
:10279000EFE9FFE03197F1F700C000002150310967
:1027A000F4CF929FB001939F700D11249A01260FD0
:1027B000371F8991E3CFE82FF0E0E354FE4FB49048
:1027C000282F26952695269530E0F901E355FE4FF2
:1027D000E4908770F12C082E02C0F594E7940A94D7
:1027E000E2F7E0FAEE24FF24E0F8F901E356FE4FA9
:1027F000C490D12C082E02C0D594C7940A94E2F755
:10280000C0FACC24DD24C0F8F901E357FE4F04914F
:1028100010E002C0159507958A95E2F7017011271F
:10282000E114F10411F081EE44DCC114D10411F083
:1028300086EE3FDC60E070E08B2D2BDDC114D1040F
:1028400011F086EED3DCE114F10411F081EECEDC60
:102850000115110521F060E070E08CE21ADD21968F
:102860005FCFCF92DF92EF92FF921F93CF93DF93D0
:1028700000D000D0CDB7DEB7C0903A02D0903B0276
:10288000E0903C02F0903D020E94F0096C197D0935
:102890008E099F0911E0643671058105910578F173
:1028A0000E94FC09DC01CB010296A11DB11D8983A8
:1028B0009A83AB83BC838091220190912301825C37
:1028C0009D4F20912101422F50E0253010F044E02F
:1028D00050E0BE016F5F7F4F0E94543182E090E074
:1028E0000E941B30182F811551F00E94F00960934F
:1028F0003A0270933B0280933C0290933D02812FF9
:102900000F900F900F900F90DF91CF911F91FF903C
:10291000EF90DF90CF9008958F929F92AF92BF92E9
:10292000FF920F931F93CF93DF9300D000D000D07E
:10293000CDB7DEB7F62E072F80E090E00E941B3067
:10294000182F811509F460C080911401482F50E0C0
:10295000811511F041E050E0609115017091160170
:10296000625C7D4FCE0106960E94543180904E02EB
:1029700090904F02A0905002B09051020E94F00936
:10298000681979098A099B096436710581059105E1
:1029900038F48FE392E00E943D0B9E818917A1F1EC
:1029A00081E090E00E941B308115C9F180911C01EB
:1029B000482F50E0863010F045E050E060911D0156
:1029C00070911E01625C7D4FCE0101960E945431D0
:1029D0008FE392E00E943D0B9E81891320C00E94EC
:1029E000F00960934E0270934F02809350029093CF
:1029F000510285E0FE013196A9E4B2E001900D920A
:102A00008A95E1F781E00CC085E0EFE3F2E0DE01BA
:102A1000119601900D928A95E1F71111EACF80E0AD
:102A200095E0E9E4F2E0AF2DB02F01900D929A9578
:102A3000E1F70F900F900F900F900F900F90DF9194
:102A4000CF911F910F91FF90BF90AF909F908F906B
:102A50000895A1E0B0E0EFE2F5E10C94933010911D
:102A6000930210FF43C01695169516951983009191
:102A70004802C0903602D0903702E0903802F090C1
:102A800039020E94F0096C197D098E099F0964368C
:102A900071058105910510F4011719F180912A0142
:102AA00090912B01825C9D4F20912901422F50E093
:102AB000211511F041E050E0BE016F5F7F4F0E9491
:102AC000543183E090E00E941B30811559F00E9440
:102AD000F009609336027093370280933802909326
:102AE000390281E02196E8E00C94AF3010E0BECFCF
:102AF00086E090E00E9474318093930282FD07C0CB
:102B00008DE38093930283E992E00E94AE0C809162
:102B10009302803420F087708863809393029091B1
:102B20009302892F817090FF04C0892F8695869526
:102B300086950C94DD060F931F93CF93DF93863019
:102B400030F56A3020F5463010F5C42FD0E0CC0FB8
:102B5000DD1F2CE0629FC00DD11D112438E7839F3B
:102B6000C00DD11D1124CE0189960E947431082F09
:102B700010E0102F0027CE018A960E947431980130
:102B8000282BC901DF91CF911F910F91089580E00B
:102B900090E0F8CF462F672F20915A0230915B02C8
:102BA000232B81F4703F39F4403F61F48091580247
:102BB0009091590208957A3028F4463018F48630FE
:102BC00008F4B9CF80E090E00895A0E0B0E0EBEE2B
:102BD000F5E10C9494307C010091A8038091A70347
:102BE000082BC5E0D0E010E0C8010C2E02C095957E
:102BF00087950A94E2F780FD09C02197A8F7D12CA8
:102C00008D2DCDB7DEB7E7E00C94B030DC2EB701E8
:102C10008C2FC0DF0E94C605019779F3F1CF0F9387
:102C20001F93CF93FC01858100811181811581F073
:102C3000611571F0C801C9DFC82F682FC8010E9453
:102C40000C04B8018C2FA6DFCF911F910F9108952E
:102C5000C8010E944204C82FF4CFCF93DF93D82F2E
:102C6000C92FB3DF6D2F7C2F95DF0E94C605DF9142
:102C7000CF910895FC018481811599F08081918123
:102C8000ECDF282F92959F70963099F060F4925F58
:102C90009F70923030F4203FB1F038F481E0283E4C
:102CA00038F080E008959A5FF3CF81E0243FC9F7C0
:102CB000089591E0213F09F090E081E0283E08F07E
:102CC00080E0892B089581E00895382F292FCB01CA
:102CD000A32FB22F87369105A105B10520F48756A1
:102CE0009C4F0C94743180E0089585E290E00E943E
:102CF00074318F3289F486E290E00E9474318B3611
:102D000059F487E290E00E94743191E0873609F02F
:102D100090E0892F8170089580E0FCCFAAE0B0E0B8
:102D2000E4E9F6E10C948E30C0903302D090340286
:102D300081E090E09093340280933302812C912CB7
:102D4000E12C5401F12C15C0F80125913591472D46
:102D50006F2D8E2D0E94CA0C0E5F1F4F739486E05C
:102D60007812F2CF96E0A90EB11CF394EAE0FE16B9
:102D700039F08501000F111F04501D4F712CE4CF55
:102D8000E394FCE38F0E911C86E0E812DACF1A82FE
:102D900019821C821B821E821D8218861F8288EC6B
:102DA00090E09A87898709EF12E0FE0131967F0152
:102DB0004AE050E0B801C7010E94AE31065F1F4FE4
:102DC00057010934F3E01F0799F789E0F7011192E1
:102DD0008A95E9F78FEF9FEF9E838D8387E08A873F
:102DE0004AE050E0B801C5010E94AE31065F1F4FB6
:102DF0000939F3E01F07A1F7D0923402C0923302E1
:102E00002A96EDE00C94AA30AAE0B0E0EAE0F7E1FF
:102E10000C9491300AE912E089E4E82E83E0F82E60
:102E200097E0B92E26EFC22E21E0D22EAA24A39439
:102E30004AE050E0B701CE0101960E946431F801EA
:102E40003896DF018B2D1D928A95E9F789819A8149
:102E5000D80111969C938E938F8112968C93129722
:102E60008D8113968C931397888514968C93149761
:102E7000898515968C9315978B819C8117969C93C9
:102E80008E9316978A8587FD04C01E96DC92CE929B
:102E90001D9780FF02C0F801A08681FF07C0D801FE
:102EA00018969C911897926018969C9382FF04C084
:102EB000F80190859460908783FF07C0D801189629
:102EC0009C911897986018969C9384FF04C0F80111
:102ED00090859061908785FF07C0D80118968C91E6
:102EE0001897806218968C93BAE0EB0EF11C015F84
:102EF0001F4FE9E9EE16E3E0FE0609F099CF2A96A6
:102F0000EAE00C94AD30282FCB01283070F44AE071
:102F1000249F90011124B90167507D4F4AE050E091
:102F20000E94643180E090E008958FEF9FEF089554
:102F3000AAE0B0E0EEE9F7E10C9499309C019755D6
:102F40008115914068F4BE016F5F7F4F822FDBDFF8
:102F5000892B31F489859A852A96E2E00C94B53064
:102F600088EC90E0F9CFA0E0B0E0E9EBF7E10C9459
:102F70009430162FD72FC42FD22E8115A1F0409355
:102F8000A1030E94D7089093DA018093D901C770FA
:102F900081E001C0880FCA95EAF791D9CDB7DEB7B5
:102FA000E7E00C94B0309091A103491335C0E09054
:102FB000D901F090DA010E94D7089C012E193F092F
:102FC0007901812F9D2FB4DFE816F90628F5D0E2AC
:102FD000DD0DCD1591F0C77011E0812F01C0880F74
:102FE000CA95EAF772D9D83040F48D2D877001C0A8
:102FF000110F8A95EAF7812F62D960E070E0802F87
:1030000048D9D83058F62D2D277081E001C0880F9F
:103010002A95EAF75AD9C2CFC77081E001C0880F5C
:10302000CA95EAF7F7CFACE0B0E0E9E1F8E10C943B
:103030008A307C01DC0114968C91811509F4F4C06E
:1030400061E0C701ECDD8C01F7018581811521F17B
:1030500080919D0390919E030097F1F00817190746
:10306000D9F0FC01FF27887F9927892B09F089C0B7
:10307000A4E0EE0FFF1FAA95E1F7E35EFC4F858108
:103080008460858311830083CF015DD91092A903E9
:1030900061E0C701C4DD8C010034F2E51F0709F4CB
:1030A00083C008F071C0043232E5130709F49CC0F4
:1030B000053242E5140709F4A0C0033252E51507B2
:1030C00009F481C0D70115968C91811509F488C146
:1030D000C80197578038910508F033C1003108F0D6
:1030E00093C066E670E080E090E0EFDD81118CC077
:1030F000812C912C540101119FC004E09E012F5F8F
:103100003F4F6901D601E02F1D92EA95E9F72401AE
:103110003501FFEF4F1A5F0A6F0A7F0AC501B4013C
:10312000D4DD8983811509F46FC0813009F006C1AF
:10313000A50194012E5F3F4F4F4F5F4F2D833E837C
:103140004F835887C301B201C0DD182F8A838115D0
:1031500009F45AC08FEF810F833008F084C06D816D
:103160007E818F819885B1DD8B83811511F0C60139
:10317000D0DA2401350133E0430E511C611C711C6F
:10318000A0C0E0E0F0E07BCF013482E51807A9F0B1
:10319000023492E5190709F095CFD70115968C9165
:1031A000811591F182E006C0D70115968C918115A9
:1031B00059F180E00E949B0C27C0F70185818115A1
:1031C00019F181E0F7CFF7018581811549F083E09E
:1031D0000E94F40345E064E083E00E94760414C09A
:1031E00083E00E94FE03F6CFD70115968C918115DE
:1031F00011F084E0EDCF84E0F4CFF70185818115F3
:10320000B9F085E00E94F4038091AA0387708115CC
:1032100059F0F7018581811539F08091F10382FF22
:1032200003C082E00E949F042C96E1E10C94A6303A
:1032300085E00E94FE03E8CFB7E68B169104A10457
:10324000B10411F3C501B40140DDEFEF8E1A9E0AFF
:10325000AE0ABE0A8111F0CF01504DCF4D805E8085
:103260006F8078842EC08BEF810F833098F5240116
:10327000350143E0440E511C611C711C6D817E813F
:103280008F81988522DD8B838115D9F0C301B2012E
:103290001CDD8C83811571F08B819C8181305FEF07
:1032A000950710F0982F8827163071F0173079F0B5
:1032B0000E941C252401350134E0430E511C611C81
:1032C000711C530142011ECF0E94C924F3CF0E94FA
:1032D000EA24F0CF143009F0C1CF6D817E818F8157
:1032E0009885F3DC182F2401350184E0480E511C29
:1032F000611C711CC501B4016D5F7F4F8F4F9F4FE3
:10330000E4DC111509F480CF811509F47DCF8150DB
:10331000990B4FEF489F9001499F300D1124A12F29
:10332000A150BB0B2A0F3B1F2150310950F2EFE98E
:10333000FFE03197F1F700C00000F6CFC601E9D9F0
:10334000C0CF033028E7120709F4B0C070F5013090
:1033500048E7140709F4A8C0023058E7150709F434
:10336000D4C0011588E7180709F496C0023AF2E5BF
:103370001F0709F06CC021EE30E02770332781E091
:1033800090E001C0880F2A95EAF7209197023091CA
:103390009402311509F408C1F7013581311509F49A
:1033A000FEC0282B209397022FCF043098E71907EF
:1033B00009F48CC00530A8E71A0709F4B8C0033730
:1033C000BCE71B0799F6F7018581811509F41CCF2D
:1033D00080919402811509F4BCC00E947E1114CF23
:1033E0006801B7E5DB1AC114E1E0DE0640F769E8E1
:1033F00072E08C2D88DD892B21F5C601E4E0880F71
:10340000991FEA95E1F7FC01E35EFC4F2281213030
:1034100081F52091890230918A02232B91F020912D
:103420008B0230918C02232B61F020918D02309120
:103430008E0240918F0250919002242B352B232B2A
:1034400001F1D70115968C91811509F48FCF033ABC
:1034500022E5120708F08DC0C801905281159042F4
:1034600008F48EC0013E110509F485CF053E110513
:1034700083C0223031F720918D0230918E02232BB0
:1034800001F3FC01EE5DFC4F20812E7F2083835EE3
:103490009C4F0E94A311D5CF87E00E946F0783E95C
:1034A00092E00E94AE0CB0CE80E0F7CF8091930204
:1034B000883028F188508093930291E0883008F496
:1034C00090E08091930290FB80F913C09091930259
:1034D000892F869586958695983340F48F5F880F5F
:1034E000880F880F9770892B8093930280919302A5
:1034F00081608093930283E992E00E94AE0C8091F8
:1035000093028695869586950CC08091930280FFE4
:103510000BC08E7F8093930283E992E00E94AE0CF1
:1035200080E00E94DD0670CE0E94B40C6DCE8091CA
:1035300093028695869586958F5F8F71883008F007
:1035400080E0880F880F880F909193029770892BE5
:10355000B2CF1092A5030E94C8040E94D7088857D2
:103560009C4E909396028093950281E08093940202
:103570004BCE023B42E5140741F525EE30E0FDCE8F
:10358000D70116968C91803100F5812F99278F7184
:1035900099278230910509F4EECE4297EDCF8095C0
:1035A00082238093970230CE322F3823311569F071
:1035B000982F90959223909397020E94C004D70170
:1035C00015968C91811509F41FCE80919402811576
:1035D00009F467C0C090A503D090A4030E94D70847
:1035E00088579C4E9093960280939502F7018581AF
:1035F000811509F456C08D2D8C298D79811184C0D7
:103600000115F0E51F0700F5011520E4120708F089
:1036100082C0063E110509F444C0C80190528115CC
:10362000904208F07FC0D70116968C91803108F443
:1036300063C0C80199271092A9038D329105E9F45E
:1036400082E08093A90372C0003EB2E51B0708F038
:1036500046C0003CE2E51E0720F5003AF2E51F07F0
:10366000E0F4003622E51207E0F4C80192558034F8
:103670009105B8F01092A903C8018E32910508F0A7
:1036800062C08832910508F04FC08E31910508F074
:103690004DC004974A97A0F237C0043B32E51307A8
:1036A00049F7F7013580311409F457C00E35FCE7AE
:1036B0001F0709F44EC00F352CE7120751F00D35E6
:1036C0003CE7130709F049C080913101811509F4E5
:1036D00040C01092310180E00E94C81195CD093799
:1036E0004CE7140728F407375CE71507D0F6C2CF7C
:1036F0000B378CE71807D4CF812F8F71843189F273
:10370000863111F41092A9030E947E1180919702D4
:103710000E94BA04C6CFD70116968C91803108F06A
:1037200088CFBFCFC80187CF8A9771F78091970262
:10373000811531F08091A90392E089278093A90334
:103740000E94080DAECF8C34910581F38D329240EA
:10375000ECCF81E08093310157CD8091310181110F
:1037600069C0C80197558115914008F0FFC0580104
:10377000F8EFAF22BB24A114B10409F045CDF80144
:10378000FF2754E0EE0FFF1F5A95E1F79F01235EDC
:103790003C4F6901D70115968C91EE5DFC4F9081ED
:1037A00080FB90F99083811509F4D9C10E94D70854
:1037B0009093A00380939F03F60182818F5F8283A1
:1037C0008091A9039091A503892B83838091A40301
:1037D00084834681578166857785C6010E944708A4
:1037E000D60115968C9181FF5801B0929E03A0924C
:1037F0009D03D70115969C91911509F401C610926D
:10380000A103980130572332310508F007C684E040
:1038100090E00E947C319093F1038093F003F801D3
:10382000E150F047E232F10508F0E1C1EC51FE4C05
:103830000C941831380150EE651A71085090A603A7
:103840008091A503582A8091A403582A88E068161D
:10385000710408F05EC098012770332781E090E082
:1038600001C0880F2A95EAF7311409F44FC0582A8D
:10387000D7018D919C910E94420421E030E0F90132
:1038800002C0EE0FFF1F8A95E2F7FC87EB872091BD
:103890001303309114033E832D8340911B035091F9
:1038A0001C035A8749876AE9C62E62E0D62EA12CEE
:1038B000B12C511005C0D60112968C9181111BC0FC
:1038C000F601838190E02B853C8582239323892B0D
:1038D00091F08085982F9770911101C087E038E0B2
:1038E0006316710408F066C0311409F45FC0869550
:1038F0008170811164C09FEFA91AB90AAFE0CA0EA6
:10390000D11CB8E0AB16B104A1F61CC080955822BA
:10391000AFCF311038C080911B0390911C03081762
:10392000190781F410921C0310921B0310921703C5
:10393000109218031092190310921A031092160392
:10394000109215038091130390911403009709F4CA
:1039500008CFE8E06E16710408F0EBC0652D0E94F8
:10396000AC07811103C081E00E94C811F701858175
:10397000F801E851FC47E730F10508F03ACFEA5F7B
:10398000FD4C0C94183110931C0300931B030E94F0
:10399000F0096093170370931803809319039093B1
:1039A0001A03109216031092150362CF82FB882728
:1039B00080F99FCF311409F49ECF80FF9CCFD601B0
:1039C0008D909C900815190519F4311409F493CFC2
:1039D000ED81FE81EC15FD0509F48DCFD6011D9614
:1039E000ED91FC91309721F08081811509F483CF0E
:1039F000652DC6010E94AC07811509F47CCF81E0DA
:103A00000815190509F080E0482E4320811491041F
:103A100041F0411006C0E985FA858E169F0609F02F
:103A20006ACF80E00E94C811D0921403C0921303A1
:103A300081E0809312038FE08A9DF0018B9DF00D51
:103A40001124E656FD4F85818093990241100EC0E6
:103A50008114910459F0808191819C012450310995
:103A6000213A310508F049C00E94C8088FE08A9DBC
:103A7000F0018B9DF00D1124E656FD4FC680D780D6
:103A8000C6019A9581159F4110F420EED222992407
:103A90009394C60101978F339E4708F0912C8FE0D5
:103AA0008A9DD0018B9DB00D1124A656BD4F19964D
:103AB000ED91FC911A97309731F01B966D917C91A6
:103AC00081E0099598229114A9F08FE08A9DF00178
:103AD0008B9DF00D1124E656FD4F868197810E9443
:103AE000A80380939802C60148E06416710440F46C
:103AF0000E94140A0E94080D0AC00E94F610B6CF58
:103B00000497813A910548F48C2D0E94AF08411426
:103B100009F427CE0E94080D77CB0E94080D8FE391
:103B20009CE90197F1F700C000008C2D0E9459100C
:103B3000EECFDC012D913C910217130741F43110B7
:103B400009C01092120380E00E94C8110ACE3114FD
:103B500009F407CEFC01808585FD03CEF4CFF90181
:103B60004485558566857785C9010E944708D60139
:103B700015968C9181FF3DCEC6010E9487118091E0
:103B80009D0390919E030817190709F032CE1092F9
:103B90009E0310929D032DCE06E221EE41EE6AE1D6
:103BA0007CE7E1D931CB07E225EE45EE6BE17CE71E
:103BB000F8CF06E221EE40EE68E17CE7F2CF07E2C3
:103BC00025EE44EE69E17CE7ECCF06E221EE42EE21
:103BD0006CE17CE7E6CF07E225EE46EE6DE17CE79F
:103BE000E0CF08E221E045EE6EE17CE7DACF80919C
:103BF000F00381608093F0036091F0037091F10312
:103C000084E090E00E94AA310E945E0DFDCA80917E
:103C1000F10388608093F103EFCF8091F00382601D
:103C2000E9CF8091F0038460E5CF8091F003886054
:103C3000E1CF8091F1038160EDCF8091F10382604B
:103C4000E9CF8091F0038061D5CF8091F00380624D
:103C5000D1CF8091F0038064CDCF0E945E0D809122
:103C6000F0038068C7CF8091F0038C60C3CF809150
:103C7000F1038360CFCF8091F0038E7FBBCF809123
:103C8000F103877FC7CF8091F0038D7FB3CF809101
:103C9000F0038B7FAFCF8091F003877FABCF809114
:103CA000F1038E7FB7CF8091F1038D7FB3CF8091E9
:103CB000F0038F7E9FCF8091F0038F7D9BCF80910B
:103CC000F0038F7B97CF0E945E0D8091F0038F777A
:103CD00091CF8091F003837F8DCF8091F1038C7F12
:103CE00099CF8091F003992782FF939590FB82F9F9
:103CF00090FB83F97FCF8091F103982F909590FBF3
:103D000080F990FB81F986CF9091F003892F8F7B0A
:103D100096FF80646FCF0E945E0D9091F003892F13
:103D200097FB87F9805866CF61E08EE090E00E94B3
:103D3000903162CF60E0F9CF9091F003892F8F7EB0
:103D400094FF806157CF9091F003892F8E7F90FF71
:103D5000816050CF9091F103892F877F93FF886016
:103D600059CF89E26DC389E256C30737BCE71B0709
:103D700079F00837ECE71E07A1F09801205E324584
:103D80002032310598F4911111C0802F8F7112CA21
:103D900081E0911541F00E94F40343E062E081E08C
:103DA0001CCA82E0F6CF0E94FE03F7CF4091A30326
:103DB0008091A803282F30E02095309570E02423CF
:103DC0003723232B19F048234093A3030B37FCE739
:103DD0001F0741F4911509F417CA0E94DB030E94E2
:103DE000CD0712CA003422E5120708F055C0003290
:103DF00032E5130708F057C0011540E5140750F5E8
:103E0000011550E4150708F064C0911509F47AC053
:103E10000A35BCE71B0709F4DDC008F0C2C0013059
:103E2000FCE71F0709F4D4C003302CE7120709F49C
:103E3000C9C001151C4709F065C00E945E0D8FEFD7
:103E400094E3ACE081509040A040E1F700C0000056
:103E50000E94550A9801305521153240B0F698015C
:103E600045E0369527954A95E1F7822F8F7020918E
:103E7000A30330E041E050E0082E02C0440F551F7C
:103E80000A94E2F724233523232B09F4BECF9111A2
:103E9000A6CF1092A5033ECE9801205C3245203279
:103EA000310508F0B2CF802F8F712091A30330E04D
:103EB00041E050E0082E02C0440F551F0A94E2F77B
:103EC00024233523232B09F4A0CF911509F49CC991
:103ED00086CFD70116968C91803108F096CF91113C
:103EE00011C0212F2F7081E090E002C0880F991F30
:103EF0002A95E2F72091A30330E082239323892BB4
:103F000009F082C9D70115968C911597CD90DC9058
:103F1000811509F463C0C6010E94E515182F682FAA
:103F2000C6010E940C04B601812F0E94CA150E948E
:103F3000C6058C01F701B580A680A2942FE0A222CD
:103F40008091AA038770811501F1CB2CB114F1F097
:103F5000812F807F803461F080E2800F8830A8F06C
:103F6000812F807E803221F4023078F0A11469F034
:103F70008091F10382FF09C082E00E949F0480913A
:103F8000AA038770CC24C3948111C12CE12FE29540
:103F9000EF70103C08F082C0F0E0E35FFD4C0C9441
:103FA00018310B354CE71407B9F08091F103002468
:103FB00082FF0394802D0C351C4709F0A3CF0E948B
:103FC000F10CA0CF6FEF7FEF80E090E00E94AA316C
:103FD0000E94810D81E0F3CF80E0F1CFC6010E9405
:103FE0004204182FA0CFF12FFF70DF2E103118F0F0
:103FF000D29490EFD922B114A9F0D11459F080E2F3
:10400000800F883010F0011107C08D2D0E94BA0476
:104010000E94080D802F40C08091A9038D298093B4
:10402000A903F6CF802F0E94F610D114B9F180E2D7
:10403000800F883010F0011104C08D2D0E94C00443
:1040400006C0D0948091A9038D218093A9030E947A
:10405000080D24C0212F2F70D22E107F103219F09E
:10406000D29480EFD822011549F0013009F483C0C1
:10407000B11409F48FC0A114A9F1CCCF8091F10340
:1040800082FD2CC0B11421F1D11429F08D2D0E9494
:10409000BA040E94080D80E00E945910C11409F46E
:1040A000D9C08091AA0380FDD5C0D70115961C9276
:1040B0008695869586950E94F403C7010E94131881
:1040C0008091AA038695869586950E94FE03C2C0BC
:1040D00080E00E94F610D11409F3AFCFB11469F15A
:1040E000A11004C08D2D0E945F11D8CF31E0A31222
:1040F00010C01091A4038D2D8123D81679F20E944F
:10410000D7089093AE038093AD031D291093A403A9
:10411000C5CF45E0A412C2CF8D2D0E945F118D2D19
:104120000E94F7088091A6039D2D9823D91609F4C3
:10413000B5CF8D298093A603B1CFA11012C08D2DCC
:104140000E9465118D2D0E94F7088091A6039D2D78
:104150009823911509F4A2CFD094D822D092A60327
:104160009DCF51E0A5129ACF8091A5038D21811595
:1041700009F494CFE4CFB11429F086E0A81608F032
:104180008DCFB0CF95E0A91608F088CF8D2D0E9475
:10419000651184CFA114D1F3093349F4AFEFB7EE21
:1041A000E3E0A150B040E040E1F700C00000802F04
:1041B0000E94F61073CF812F8695869583708115A6
:1041C00061F0813009F06ACFC8019370B11002C06C
:1041D00080E090E00E94870861CFC8019370B11021
:1041E00002C080E090E00E945F0858CF6B2D802FC6
:1041F0000E94350953CF812F8370811139C0B110CE
:1042000027C0402F429546954770440F440F802F9A
:104210008F70042E01C0880F0A94EAF7202F2071B6
:1042200004FF07C02FE030E001C0220F4A95EAF7F3
:1042300020951695169513701230A9F0133089F059
:104240003091A703113061F0822B83230E94EE038B
:104250000E944C0860E0C7010E940F160C941419CC
:10426000832B822BF3CF822B9091A7038927EECF4C
:10427000B11451F110FFECCF402F42954695477095
:10428000440F440F802F8F70042E01C0880F0A94B2
:10429000EAF7202F207104FF07C02FE030E001C0B3
:1042A000220F4A95EAF7209516951695137012304D
:1042B00089F0133069F03091A803113041F0822B5E
:1042C00083230E94F103C4CF823010F2D5CF832B19
:1042D000822BF7CF822B9091A8038927F2CF1F70F2
:1042E000B11439F0812F0E94F403802F0E945F11D6
:1042F000AFCF802F0E946511812F0E94FE03A8CFAF
:10430000023F71F170F4003FC9F0013F91F0B11428
:1043100009F465C0A11409F45FC0802F0E945910F0
:1043200097CF033F21F1043F91F78091F10382FD84
:104330002AC0812F8F71B11401F316C0B11469F036
:10434000F5E0AF1608F084CF1F7181E090E0012EF8
:1043500001C0880F0A94EAF7BECF26E0A216F2CF7A
:10436000812F8F71B110C9CF0E94F40371CF80E00B
:10437000B11409F4A6CF1F7181E0012E01C0880F8E
:104380000A94EAF79ECFB114C1F08091AA03877016
:10439000843049F41092AA031092AC031092AB033C
:1043A000812F8F71AACF35E063E0A31608F050CFBC
:1043B000812F8F710E94E3084BCF45E0A41640F097
:1043C0001092AA031092AC031092AB0364E0F0CFFA
:1043D00081E00E949F043CCF812F8F71C5CFA11433
:1043E000F9F2093349F45FEF87EE93E051508040D2
:1043F0009040E1F700C00000802F0E94F61028CF07
:104400000631BCE71B0709F0B0CC8091A2038115EF
:1044100009F4A9CC85E30E94C8087CCB0631ECE7FF
:104420001E0709F0A2CC8091A5038A7A91E0811140
:1044300001C090E09093A203811509F492CC85E32A
:104440000E94AF0867CBA0E0B0E0E9E2F2E20C9492
:1044500094308091EF03803108F049C08091EE03E1
:10446000811509F444C0C091B00387E0D82E809133
:10447000AF038C17E1F1EC2EF12CDC9EE00111244E
:10448000FE01EF54FC4F84818115B1F1918180913F
:10449000EA03981331C090818091E90398132CC0EE
:1044A0008581811129C0028113818091EB03909154
:1044B000EC03081B190B60E089EE93E00E940F16D5
:1044C0000E94981708171907B8F48091EF038F70AE
:1044D00080618093EF03C954DC4F88818F708061C5
:1044E000888389EE93E00E9413180E949504CDB74B
:1044F000DEB7E7E00C94B030E7012196C770B7CF84
:10450000ADE0B0E0E6E8F2E20C948C308C0186E09D
:10451000F801DE01189601900D928A95E1F7F801F5
:10452000F580E48089EE882E83E0982E8091ED035B
:10453000811117C0E11491F0F11409F455C1C801BB
:104540000E943A16811509F44FC187E0F801A9EEDF
:10455000B3E001900D928A95E1F775DFFF24F394A3
:1045600061C0A280B380D090EE038091EB03909164
:10457000EC033501681A790AD11409F4F0C0C0803F
:10458000518060E089EE93E00E940F160E94981718
:104590006816790608F09EC0E11401F38091EA03E1
:1045A000F8019181E090EF03F0E1EF1608F05BC0B5
:1045B000981317C09091E903F8018081981311C0F6
:1045C000F1104BC08E2D8F7080618093EF0389EEC8
:1045D00093E00E9413188091EF03F8018683F12C79
:1045E00021C0F1103AC040E0652D8C2D0E94E00BF7
:1045F00040E0652D8C2D0E94E00BF82E8111EFCF4D
:10460000888599850E942D16292F22952F70903428
:1046100070F49F702230A0F09115B1F0F8019681EE
:10462000903190F48F2D2D96EFE00C94A8302A5FF6
:104630002F70223068F0C8010E941318FD2CF2CFB1
:10464000911511F0811571F3805E883058F3F3CF26
:10465000803F40F3815F8330F9CF8091EF03816029
:104660008093EF03BCCF981315C09091E903F80134
:10467000808198130FC0F1100DC0E682C8010E941E
:10468000131887E0F801A9EEB3E001900D928A9526
:10469000E1F764CFC8010E943A16811509F4A4C05D
:1046A000F11409F4A1C08091EF03803208F44DCFDA
:1046B0008091E9039091EA039A838983BC82AB825B
:1046C0008091ED038D831E82EF82CE0101960E94C0
:1046D00013183BCFD090EF03F0E1DF1650F489EED2
:1046E00093E00E94131887E0F40111928A95E9F78C
:1046F00076CFE11409F432CF9091EA03F801818179
:10470000981311C09091E903808198130CC0F110A7
:104710000AC0D682C8010E94131887E0F4011192E2
:104720008A95E9F71BCFC8010E943A16811509F452
:104730005BC0F11409F458C08091EF03803208F493
:1047400004CF8091E9039091EA039A838983BC8224
:10475000AB828091ED038D831E82DF82B6CF60E055
:1047600089EE93E00E940F160E949817681679064A
:1047700008F0B9CFE11409F4F1CEF114A9F1909148
:10478000EA03F8018181981325C09091E9038081A3
:10479000981320C08091EB039091EC03A81AB90AFA
:1047A000F8ECAF16B10408F06CCF8091EF0380FDF8
:1047B00068CF803108F465CFF8018683982F907F09
:1047C000903F09F45BCF982F907F905F8F70892B7B
:1047D000868354CFC8010E943A168111B6CE8091CB
:1047E000EF0381608093EF03C8010E941318B6CED7
:1047F000ABE1B0E0EEEFF3E20C9497304E8B5F8BC1
:10480000688F798F8A8F192F9B8F91111092A9032E
:104810001D8A86E0FE017696DE011F9601900D92BC
:104820008A95E1F70A8D8091F10382FF1FC00E94F3
:10483000D7082091AB033091AC03821B930B8838CF
:10484000934138F08091AA0382FD03C082E00E9468
:104850009F040E94D7082091AD033091AE03821BC4
:10486000930B8838934110F00E94C804011561F041
:104870000B8B1C8B61E0CE010F960E940F1661E03E
:10488000CE010F960E940F160B8B1C8B87E0FE014A
:104890003F96DE01189601900D928A95E1F7CE01C0
:1048A00008962EDE811110C02091AF033091B00325
:1048B00087E0FE013896DE01119601900D928A95EF
:1048C000E1F78C8581110BC017E08091B0039091C6
:1048D000AF0389132BC06B96E4E00C94B330822FA6
:1048E00090E00196877099273817190671F40E9495
:1048F0005E0D1092AF031092B00387E0E9EEF3E093
:10490000DF011D928A95E9F7DFCF97E0929FD001F2
:104910001124AF54BC4FFE01319601900D929A952F
:10492000E1F78093AF030E949504CECF189FC0019A
:1049300011248F549C4FE4DD811569F28091B003FE
:1049400090E00196877099278093B003BECFA6E0D0
:10495000B0E0EDEAF4E20C9497300E94D7088C01A5
:1049600080915C0290915D028017910771F019822D
:104970001A820E94D708BC0149815A8180E090E0E8
:1049800037DF10935D0200935C022696E4E00C94FE
:10499000B330A6E0B0E0EFECF4E20C9499309093E1
:1049A000590280935802811520E2920730F40E9448
:1049B000E1102696E2E00C94B53080EF89838A837B
:1049C0000E94D7088160BC0149815A8181E091E051
:1049D0000FDFEFCFA6E0B0E0E0EFF4E20C94973009
:1049E0008C019093590280935802011580E21807B8
:1049F000B0F4802F0E94F610C801805E91090897DC
:104A000028F064E771E10115110511F465E671E123
:104A1000C8010E94D2032696E4E00C94B33080EFE4
:104A200089838A830E94D7088160BC0149815A81A9
:104A300081E090E0DDDEEFCFCF93DF93D82FC92F59
:104A4000A8DF8D2F9C2FC6DFDF91CF9108950F93A4
:104A50001F93CF93DF938C01862F69E872E00E9449
:104A60008317892B91F4C0918902D0918A022097F3
:104A700061F0F8018281833039F4CE01DDDFCE01AF
:104A8000DBDFCE01D9DF01C0E0F7DF91CF911F91CD
:104A90000F9108950F931F93CF93DF938C01EB0138
:104AA00069E872E08C2F0E948317892B09F057C0A8
:104AB000FE01FF27D80112968C911297E950FE4F04
:104AC0008130A9F415968C9182FD4EC080FF4CC0B8
:104AD00082E0808380918B0290918C020097B9F4E0
:104AE0008091890290918A020097C9F110C08230AA
:104AF000A1F515968C9182FD26C080FD0AC083E049
:104B0000808380918D0290918E020097F1F041DFB9
:104B100026C084E0808380918F029091900200975C
:104B2000B1F78091890290918A02009701F184DFA8
:104B300080918B0290918C02009749F780918902B5
:104B400090918A02E4CF85E08083809189029091E0
:104B50008A02009721F070DFF1CF86E08083DF9139
:104B6000CF911F910F91089581E08083B9CF8091FB
:104B70008B0290918C02B8CF0F931F93CF93DF934A
:104B80008C01EB0169E872E08C2F0E948317892B5E
:104B900071F4DD27C950DE4F8881F8011282188236
:104BA0008330E9F048F4813059F0823081F0DF91B0
:104BB000CF911F910F9108958430B1F08530B9F7EE
:104BC0008091890290918A02009789F306C08091B2
:104BD0008B0290918C02009799F3FCDEE8CF8091D4
:104BE0008D0290918E02F7CF80918F02909190026A
:104BF000009799F72091890230918A0280918B0267
:104C000090918C0221153105F9F2009731F7C90115
:104C1000E4CFA0E1B0E0EFE0F6E20C948B30FE01CF
:104C2000319680E1DF011D928A95E9F707E010E0F7
:104C300099E9A92E93E0B92E27E6422E512C612C3A
:104C4000712C4F0173016201B1E14B1651046104F3
:104C500071041CF080E1C82ED12CA601B501C4015D
:104C60000E948131AC0CBD1C0D2C000CEE08FF081D
:104C70004C185D086E087F080150104019F76096C7
:104C8000E0E10C94A7306FEF85E290E00E94903154
:104C90006FEF86E290E00E9490316FEF87E290E044
:104CA0000E94903160E088E290E00E9490310E9482
:104CB0008E16AFDF6FE285E290E00E9490316BE6E6
:104CC00086E290E00E94903167E687E290E00C94E3
:104CD0009031CDB7DEB7AC970FB6F894DEBF0FBEFC
:104CE000CDBF85B7806885BF85B7806885BF84B72D
:104CF000877F84BF0FB6F894A89580916000886183
:104D000080936000109260000FBE80E890E00FB6C4
:104D1000F89480936100909361000FBE81E08093CE
:104D2000030182EC96E09093C5018093C4010E9438
:104D300094070E9404170E94100B0E94860B80911A
:104D4000E20084608093E2007894809135028115BE
:104D500099F08091E9001091EC008F701795112760
:104D60001795182B1092E9008091E80083FD0E94AE
:104D7000960D1F701093E90082E084BD93E095BD0D
:104D80009AEF97BD80936E001092540210925502D4
:104D900010925602109257020E947516811101C09E
:104DA00072DF8091D80080618093D8002AE12A9533
:104DB000F1F700C08091D900182F117080FD04C058
:104DC0000E94100B1092350210935202109353025E
:104DD0001093040111110E94362F809104018091DB
:104DE000040190E0811101C095E090930A0285E0F2
:104DF000891B809309020AE411E0D8018D918D018D
:104E00008F3F11F00E94C406B1E00F341B07A9F7D1
:104E10000FE411E055E5E52E51E0F52EF801819102
:104E20008F018F3F11F00E94C406E016F106B1F722
:104E30008AE0E9E2F2E0DF01282F1D922A95E9F7E6
:104E4000EFEFF1E0DF011D928A95E9F780E090E055
:104E50000E947C31833E9E4F21F40E947516811181
:104E600036C063EE7EEF80E090E00E94AA3160E001
:104E700082E090E00E94903181E08093A70361E09E
:104E800083E090E00E94903160E074E184E090E083
:104E90000E94AA311982CE0101960E94AE0CF3DE67
:104EA0000E94B40C85E00E946F0783E992E00E94A3
:104EB000AE0C40E050E0BA018FE090E00E94A231D9
:104EC00040E050E0BA0183E190E00E94A23182E02C
:104ED00090E00E94743180930D0284E090E00E9483
:104EE0007C319093F1038093F0030E942312EFEF43
:104EF000F6E721E0E150F0402040E1F700C000007B
:104F00000E9423128091290280FF08C06FEF7FEF7B
:104F100080E090E00E94AA310E94550A83E090E070
:104F20000E9474310E94EE03269A2E9882E28093AA
:104F3000800089E1809381008FEF9FEF909387003D
:104F4000809386000E9478150E9478158091520205
:104F5000811101C08ED785E091E090935F0280932C
:104F60005E0280913502853059F48091350285309A
:104F700009F452C00E945E0D0E9478150E944C08F0
:104F80000E9423120EE012E049E2E42E42E0F42EE9
:104F9000D701F80191918D9128E132E02E173F075A
:104FA00009F471C09817B1F380905202D12CD70147
:104FB000CD907D01F80191908F019C1431F19C24DA
:104FC000B12CAA24A394892D8A218115B9F08114CA
:104FD000A9F0B982DA820E94D7089C838B83F1E022
:104FE000FD8391E08C2D8A21811101C090E09E8388
:104FF00049815A816B817C818D81FADBB394AA0C43
:1050000026E0B212E0CFF801C292D3943AE0D31274
:10501000CECF0E94FC093AC080913502843039F12C
:1050200080E00E946F0710920B0288E190E0A0E4FC
:105030000FB6F894A895809360000FBEA09360000F
:1050400083B7817F846083BF83B7816083BF789497
:10505000889583B78E7F83BF0FB6F894A89580910B
:105060006000886180936000109260000FBE0E9413
:105070002312E9E2F2E0819181110AC5B2E0E33343
:10508000FB07C9F772CF98138FCF61DC8091520272
:10509000811509F478C000911503109116030115CC
:1050A000110591F1C0901C02D0901D02E0901E02EB
:1050B000F0901F020E94F0096C197D098E099F096A
:1050C000C0901802D0901902E0901A02F0901B02D2
:1050D0006C157D058E059F05B8F0C8010E94E11092
:1050E000109215031092160310921C0210921D02CA
:1050F00010921E0210921F021092180210921902B2
:1051000010921A0210921B02E0909D03F0909E03F1
:10511000E114F10439F1C0909F03D090A0030E94E4
:10512000D7088C010C191D09C7010E949817801718
:105130009107C0F420919D0330919E03C9019927E6
:10514000287F3327232B09F02FC134E0880F991FC4
:105150003A95E1F7835E9C4FDC0115962C9122FF76
:105160000E94A31180919402811569F00E94D708D2
:105170002091950230919602821B930B8F3F9F479F
:1051800010F40E947E1186E0E3E8F2E0DE01119661
:1051900001900D928A95E1F7B0908402D09085023B
:1051A000F0908602C0908702E090880210928502FB
:1051B0001092860210928702109288028F2D8D29FC
:1051C000811509F441C000912202109123020E942E
:1051D000D7089C01201B310B90918102911509F495
:1051E00052C42531310580F19F3F19F09F5F9093A4
:1051F0008102D11459F00E94020891E01D140CF0B4
:105200009FEF899F802D112480938502F11459F01E
:105210000E94020891E01F140CF09FEF899F802DDF
:1052200011248093860280918502811569F0109186
:105230008602111549F00E94F40780938502812FA0
:105240000E94F407809386028C2D8E29811509F423
:1052500041C000912002109121020E94D7089C01B8
:10526000201B310B90918002911509F407C4213560
:10527000310580F19F3F19F09F5F90938002C11428
:1052800059F00E94220891E01C140CF09FEF899FB6
:10529000802D112480938702E11459F00E94220886
:1052A00091E01E140CF09FEF899F802D11248093B4
:1052B000880280918702811569F01091880211158A
:1052C00049F00E94F40780938702812F0E94F4071F
:1052D00080938802809184028B1119C0809185028D
:1052E000811511F08D1113C020918602211511F046
:1052F0002F110DC090918802911511F09E1107C0D9
:1053000030918702311103C0822B892B81110E94B9
:105310000C0986E0FE013196A3E8B2E001900D92FF
:105320008A95E1F70E944C0890912402891721F098
:10533000809324020E94F00980913502843009F0A4
:1053400010CE83E08093E9008091E80082FF09CECF
:105350008091E80090E085FF05C00E94DF0A81157A
:1053600031F191E08091E8008B778093E80091150E
:1053700009F4F7CD00915A0210915B02E981011501
:10538000110589F1EE3F09F050C08A81833020F089
:105390008550833008F049C0EA81EE3008F045C0FE
:1053A000F0E0E75EFD4C44C780E090E0D5CE00E23F
:1053B00010E0FE0131967F018091E80085FD0AC072
:1053C0008091E8008B778093E8000E94DF0A8115C6
:1053D00099F3C7CF8091F100D7018D937D010150E2
:1053E000104051F7BECFE43148F4E11549F0E150E7
:1053F000E33130F4F0E0E95DFD4C1AC7EE3F61F2B5
:105400008FEF898312C01A8289E08B830EC08A8154
:10541000823081F08330B1F0813091F70E94F00941
:105420000DD76B837C838D839E83CE0101960E9472
:105430002F0B97CD88E290E057D71B821C821D82EC
:105440008E83F3CF8091330290913402892B69F3DC
:105450008AE0E9E2F2E0DE01139601900D928A956E
:10546000E1F7E3CF8A81823059F66B817C818D81AF
:105470009E81E4D688E290E053D7D7CF4C816B81F0
:105480008A810E949B159827892798279E838D8360
:10549000CCCF2D813E813227232732274C816B814F
:1054A0008A810E94CA0CC1CF0E948E16BECF8A810B
:1054B000893009F0BACF8B81B7E08B9FC0011124EE
:1054C0006FEF70E06CD6862F0E946F07AECF8A8197
:1054D000893029F08A3009F0A8CF1B82A6CF8091AD
:1054E0009302869586958695EFEF8E9FC0011124D5
:1054F00067E070E054D66B8398CF83E992E00E9416
:10550000AE0C93CF80E18A8390CF1A8287E67DCF5D
:105510008C818D3108F089CF8A809B8098248924E2
:105520009824A12CB12C8E010F5F1F4F7801E80E3B
:10553000F11C0E151F0509F478CF80E0F7E68F16F1
:105540009104A104B10420F4C40187569C4FCCD629
:10555000D80114968C930F5F1F4FBFEF8B1A9B0AD5
:10556000AB0ABB0AE6CF8091330290913402892BBB
:1055700009F45BCF8C818D3108F057CF882E912CA8
:10558000A12CB12CCA80DB80DC24CD24DC24E12CCE
:10559000F12C8E010F5F1F4F412C512C320148140A
:1055A00059046A047B0408F040CFE7E6CE16D10424
:1055B000E104F10438F4D80114966C91C6018756C1
:1055C0009C4FAED6BFEF4B1A5B0A6B0A7B0AEFEF1C
:1055D000CE1ADE0AEE0AFE0A0F5F1F4FE0CF19DB7C
:1055E00024CF86E090CF8C818D3108F01ECF882E9D
:1055F000912CA12CB12CCA80DB80DC24CD24DC24AE
:10560000E12CF12C412C512C32018E010B5F1F4FEC
:10561000481459046A047B0408F007CF80E0F0EDD9
:10562000CF16F2E0DF06E104F10418F4C601899612
:105630005BD6D8018D938D01BFEF4B1A5B0A6B0AC5
:105640007B0AEFEFCE1ADE0AEE0AFE0AE1CF2C81CA
:10565000022F10E02D3108F0E8CE8A819B81982737
:10566000892798272C01612C712C803DF2E09F073F
:1056700008F0DBCE822E912CA12CB12C40ED52E013
:1056800060E070E044195509660977094217510531
:105690006105710508F4C9CE2091330230913402BE
:1056A000232B09F03EC01C0129E2220E311C80FB95
:1056B000EE24FF24E0F880FF0BC0889615D69D816C
:1056C00089279827892781159C4711F48FEF8D83AF
:1056D000D501C401840D951DA61DB71D80FF19C0FD
:1056E000680181E0C81AD108DE011596AC0DBD1D18
:1056F000BCA7ABA7C101800F911FF6D5EBA5FCA5F8
:10570000908181159C4721F48FEFABA5BCA58C93AC
:105710008601FE013196EE0DFF1D2FEFE016F1061A
:1057200038F08E010F5F1F4FC12CD12C760125C0A0
:105730009481858181159C4711F42483258332E06F
:10574000E30EF11C3296EACF80ED481682E058064F
:105750006104710430F4D80114966C91C2018996E9
:10576000DFD5BFEFCB1ADB0AEB0AFB0AEFEF4E1ACD
:105770005E0A6E0A7E0A0F5F1F4FC814D904EA043E
:10578000FB0410F352CE8091330290913402892BA6
:1057900009F44BCECE0101960E942F0BFFEF21EEB4
:1057A00034E0F15020403040E1F700C00000B4CBBD
:1057B00088E0E2E3F1E0DE01919601900D928A9596
:1057C000E1F7FE0132968FE1DF011D928A95E9F73C
:1057D00086E0898388E07F96DE0115963ECE88E4D8
:1057E000898381E08A831B821C821FCE8B819C81EE
:1057F000092E000CAA0BBB0B25E0880F991FAA1FCE
:10580000BB1F2A95D1F7AC01BD01405E5F4F6F4FC2
:105810007F4F481759076A077B0708F406CE88347C
:10582000E1E09E07A105B10508F0FFCD4934F1E0A4
:105830005F076105710520F048E451E060E070E029
:10584000481B590BBC0164537A4FCE01019616D503
:10585000ECCD4AE150E06FEF70E0CE0107962DD518
:105860008091330289830A831B821C821D8281E01E
:10587000E7CD81E090E090935B0280935A0282E34F
:1058800090E090932802809327020E94D70890937B
:10589000260280932502C9CD0115110571F1D09022
:1058A0002902E0902502F09026020E94D7088E1966
:1058B0009F098536910540F1D1FE26C0D0FE24C057
:1058C0000E94D70890932602809325028091270298
:1058D0009091280201979093280280932702892BA8
:1058E00061F410925B0210925A0281E090E0909372
:1058F00034028093330200E010E080913302898308
:105900000A838091270281CD82E390E09093280260
:1059100080932702F2CF109234021092330285CD89
:1059200040E250E06FEF70E0CE010196C6D47DCD2D
:105930008B81823009F450C078F4811136C0FE01A9
:1059400032968EE1DF011D928A95E9F788E089831E
:105950008B8383E088A369CD853009F472C08630DB
:1059600009F063CD1C818AE0FE013596DE01919637
:1059700001900D928A95E1F78BA19CA10E94870767
:105980009CA38BA38FEF183060F4FAE01F9FB00147
:105990001124675B7C4F4AE050E0CE018196DED453
:1059A00080E089830E94041740CD8C819AE0F92E13
:1059B0008E010F5D1F4FF8012F2D11922A95E9F7E7
:1059C000B8010E9483178983F801DE0112960190C5
:1059D0000D92FA94E1F729CD1C818AE0FE013596FB
:1059E000DE01919601900D928A95E1F789A19AA125
:1059F0000E9487079AA389A38BA19CA10E94870775
:105A00009CA38BA38DA19EA10E9487079EA38DA31B
:105A10008FA198A50E94870798A78FA38FEF1830B2
:105A200060F43AE0139FB001112467507D4F4AE0C3
:105A300050E0CE01819692D480E089830E94940741
:105A4000F4CC2C816AE0CE018196DC01E62F1D9218
:105A5000EA95E9F7283080F4629FB0011124675B72
:105A60007C4F4AE050E030D480E089838AE0FE0138
:105A7000B196DE011296F1CC8FEFF7CF2B303105C6
:105A800008F0FACB27CC2B30310508F0AFCBDCCBBC
:105A900080910C02811509F468CAE0E1E9BDF2E1E8
:105AA000F9BD09B400FEFDCF8091D8008F7D8093B1
:105AB000D8008091E00082608093E0008091E00057
:105AC00081FDFCCF0E945E0D50CA1F921FB61F922F
:105AD00011248F939F93AF93BF9380910B028111F9
:105AE00013C08091EE019091EF01A091F001B0916F
:105AF000F1014196A11DB11D8093EE019093EF013C
:105B0000A093F001B093F101BF91AF919F918F915C
:105B10001F901FBE1F90189578941F921FB61F925A
:105B200011248F939F93AF93BF938091EE01909137
:105B3000EF01A091F001B091F1010196A11DB11DFD
:105B40008093EE019093EF01A093F001B093F101E7
:105B5000BF91AF919F918F911F901FBE1F9018957D
:105B60001F920F920FB60F9211242F933F934F93D2
:105B70005F936F937F938F939F93AF93BF93EF93B5
:105B8000FF938091E10082FF09C08091E20082FFD3
:105B900005C08091E1008B7F8093E1008091DA0065
:105BA00080FF24C08091D80080FF20C08091DA005F
:105BB0008E7F8093DA008091D90080FFA9C080E1B8
:105BC00089BD82E189BD09B400FEFDCF81E08093EB
:105BD00035028091DD01811109C00E94100B0E94E5
:105BE000860B8091E20084608093E2008091E10066
:105BF00080FF1AC08091E20080FF16C08091E20011
:105C00008E7F8093E2008091E20080618093E200C9
:105C10008091D80080628093D80019BC85E0809381
:105C2000350283E0809303018091E10084FF2FC05F
:105C30008091E20084FF2BC080E189BD82E189BDB3
:105C400009B400FEFDCF8091D8008F7D8093D800ED
:105C50008091E1008F7E8093E1008091E2008F7E51
:105C60008093E2008091E20081608093E200809165
:105C7000DC01811509F452C084E0809335028091E3
:105C80003502843009F052C082E080930301809194
:105C9000E10083FF2CC08091E20083FF28C0809147
:105CA000E100877F8093E10082E0809335021092CB
:105CB000DC018091E1008E7F8093E1008091E20021
:105CC0008E7F8093E2008091E20080618093E20009
:105CD00042E060E080E00E94560B8091F000886016
:105CE0008093F00081E08093030180930201FF9193
:105CF000EF91BF91AF919F918F917F916F915F9144
:105D00004F913F912F910F900FBE0F901F901895BC
:105D100019BC109235021092DD0168CF8091E3002A
:105D200087FF02C083E0A9CF81E0A7CF81E0ADCF9C
:105D30001F920F920FB60F921124EF92FF920F93C2
:105D40001F932F933F934F935F936F937F938F9303
:105D50009F93AF93BF93CF93EF93FF9309EE10E020
:105D6000F8018081C091EC008F70C795CC27C79552
:105D7000C82B108280EFE82EF12CF7018081877FFD
:105D8000808378940E94960DF8011082F70180813B
:105D900088608083CF70F801C083FF91EF91CF912D
:105DA000BF91AF919F918F917F916F915F914F9133
:105DB0003F912F911F910F91FF90EF900F900FBE89
:105DC0000F901F9018958EE1489B02C08A95E1F7CD
:105DD000489BFECF0895589880E28A95F1F7589A2B
:105DE0000895FC012BE02A95F1F728E090E080E08F
:105DF00031E040E14A95F1F7880F489B02C081608D
:105E0000932742E04A95F1F7000040E14A95F1F707
:105E10002A9579F720E12A95F1F729B132E03A95F0
:105E2000F1F7000040E14A95F1F7217092272081B7
:105E3000920F90830895A1E0B0E0E0E2FFE275C127
:105E400019828C017C01E60EF11CBDDFCE010196AA
:105E5000C8DFF80181938F01EE15FF05B1F781E0EE
:105E60009981911180E02196E6E07BC1509A589A81
:105E700008955098589AE89AE9E6F0E080818C7F7E
:105E8000808308956150770B91E001C0990F6A9566
:105E9000EAF7692F90E021E0611108C0911599F0AF
:105EA000589A80E28A95F1F758980895362F38234A
:105EB000311539F0589A922730E23A95F1F7669504
:105EC000EBCF5898F9CF5898ECCFFF920F931F93D0
:105ED000CF93DF93EC018C01060F111DF9907BDF4E
:105EE00068E08F2DCFDFC017D107C1F7CDB7DEB780
:105EF000E5E038C11F920F920FB60F9211240F9355
:105F00001F932F933F934F935F936F937F938F9341
:105F10009F93AF93BF93EF93FF93CF93DF930F9232
:105F2000CDB7DEB719824FDFCE0101965ADF082FB9
:105F3000069506950695982F92959570202F2570B9
:105F4000920F292F237096959695920F9827977008
:105F50008981892B811509F058C0053008F055C09A
:105F600080E18A95F1F7589A509A82E08A95F1F784
:105F700000C0589888E0089F80011124D801AF5EC6
:105F8000BE4F1696ED91FC9117973097A9F060914E
:105F900055017091560114962D913C911597260F3D
:105FA000371F11968D919C911297680F791F139648
:105FB0004C9113978C910995F801EF5EFE4F638128
:105FC000611549F0209155013091560184819581E8
:105FD000820F931F7ADFFFDE80E18A95F1F75898F0
:105FE0005098589A80E18A95F1F7F801EF5EFE4FDC
:105FF0006081611549F020915501309156018181F0
:106000009281820F931F17DFDEDE0F90DF91CF9119
:10601000FF91EF91BF91AF919F918F917F916F9180
:106020005F914F913F912F911F910F910F900FBE54
:106030000F901F9018950F931F93CF93DF938C01B0
:1060400005970CF05EC0F894509A589885E08A95B0
:10605000F1F70000C02FC695C570802F8570C80F5E
:106060008C2F8370C695C69593E0000F111F9A95EB
:10607000E1F7C80FC8018C2BEC01ADDE00C068E071
:106080008C2F00DF90E19A95F1F75098589A489B31
:1060900031C087E090E048992FC0F801EF5EFE4FD5
:1060A0006381611559F02091550130915601848129
:1060B0009581820F931FBFDE811501F184DE80E29E
:1060C0008A95F1F75898509A90E19A95F1F7F8016E
:1060D000EF5EFE4F6081611549F0209155013091CE
:1060E000560181819281820F931FEFDE74DE7894D6
:1060F00081E008C000C0CBCF019749F4509A589A6C
:10610000789480E0DF91CF911F910F91089500C0A6
:10611000C2CF2F923F924F925F926F927F928F9257
:106120009F92AF92BF92CF92DF92EF92FF920F9326
:106130001F93CF93DF93CDB7DEB7CA1BDB0B0FB630
:10614000F894DEBF0FBECDBF09942A8839884888ED
:106150005F846E847D848C849B84AA84B984C88483
:10616000DF80EE80FD800C811B81AA81B981CE0F7A
:10617000D11D0FB6F894DEBF0FBECDBFED0108955F
:10618000DB018F939F9370D0BF91AF91A29F800D41
:10619000911DA39F900DB29F900D11240895AA1BED
:1061A000BB1B51E107C0AA1FBB1FA617B70710F002
:1061B000A61BB70B881F991F5A95A9F78095909534
:1061C000BC01CD01089597FB072E16F4009406D06C
:1061D00077FD08D0E4DF07FC05D03EF4909581956B
:1061E0009F4F0895709561957F4F0895A1E21A2EF3
:1061F000AA1BBB1BFD010DC0AA1FBB1FEE1FFF1F6B
:10620000A217B307E407F50720F0A21BB30BE40BBA
:10621000F50B661F771F881F991F1A9469F7609501
:106220007095809590959B01AC01BD01CF010895BB
:10623000EE0FFF1F0590F491E02D09946927962732
:1062400069277827872778270895A29FB001B39FF1
:10625000C001A39F700D811D1124911DB29F700D6F
:10626000811D1124911D0895F0DFA59F900DB49F0D
:10627000900DA49F800D911D11240895FB01DC0158
:1062800002C005900D9241505040D8F70895FB018F
:10629000DC0104C08D910190801921F441505040DF
:1062A000C8F7881B990B0895FB01DC0102C001901F
:1062B0000D9241505040D8F70895DC0101C06D9314
:1062C00041505040E0F70895DC01CB01FC01F99901
:1062D000FECF06C0F2BDE1BDF89A319600B40D9232
:1062E00041505040B8F70895F999FECF92BD81BD55
:1062F000F89A992780B50895A8E1B0E042E050E00F
:10630000E5CFDC01A40FB51F4150504040F0CB0158
:10631000840F951F2E9105D041505040D8F7089515
:10632000262FF999FECF92BD81BDF89A019700B44E
:10633000021639F01FBA20BD0FB6F894FA9AF99AEE
:106340000FBE08950396272FECDFEADF252FE9DF44
:10635000242FE7CF0196272FE4DFE2CFDC01CB012A
:1063600002C02D9105D041505040D8F70895262FF6
:10637000F999FECF1FBA92BD81BD20BD0FB6F8942A
:10638000FA9AF99A0FBE01960895F894FFCF410941
:10639000460948094D095D095D095D095D095D0909
:1063A0005D095D095D094F09530956095B096B09D0
:1063B00071097509730E990E9F0E990E9F0EF10EBD
:1063C000120F9F0E181025103B1EA31E431E0D1EFC
:1063D000111E471E151E4B1E571E211E9C1E251EDC
:1063E0005B1E291E5F1E841E2D1E631E8B1E331E08
:1063F000691E711E191E4F1E1D1E531E371E6D1E57
:106400007B1E941E9A1E071E3F1EAA1ED91DDF1D4D
:10641000CC1DD31DE51DEB1DF11DF31FF31F2A201D
:106420002A20DB20F6204E204E20FB206F218021E9
:106430008021D82BEF2BF62B152A152A292C392C45
:106440004C2C8B2C902C152A152A152A982C032AB3
:10645000072A322A3E2A492A542A572A672A7D2A9D
:10646000002AC32B822A852A882AB32AEF2AF12AF6
:04647000F32A272BB9
:106474000000010001D408410C660A570C5C0C387A
:106484000C000000010000000000000005010000F5
:10649400000406000000000000010A0000000000E3
:1064A4000001BBBBAD3D7081F6410044227B490134
:1064B4002701AC004F02680288029497C6343592D3
:1064C400F5F6F731333E02E200E900EA00B500B622
:1064D40000B700CD008301CC008A01920194012110
:1064E40002230224022502260227022A02B300B450
:1064F400006F0070009F01CB019F02A002E200E93F
:1065040000EA00B500B600B700CD008301CC008AD4
:10651400019201940121022302240225022602276A
:10652400022A02B300B4006F0070009F01CB019FE8
:0465340002A00200BF
:00000001FF
